:100000000C9463000C948B000C948B000C948B006C
:100010000C948B000C948B000C948B000C948B0034
:100020000C948B000C948B000C948B000C948B0024
:100030000C948B000C948B000C948B000C948B0014
:100040000C9479010C948B000C9453020C948B004B
:100050000C948B000C948B000C948B000C948B00F4
:100060000C948B000C948B000000000024002700EF
:100070002A0000000000250028002B0000000000DE
:1000800023002600290004040404040404040202DA
:100090000202020203030303030301020408102007
:1000A0004080010204081020010204081020000012
:1000B0000007000201000003040600000000000029
:1000C0000000BC009C0311241FBECFEFD8E0DEBFB0
:1000D000CDBF11E0A0E0B1E0E6E2FBE002C0059098
:1000E0000D92A431B107D9F711E0A4E1B1E001C04C
:1000F0001D92A63BB107E1F710E0C6ECD0E004C0CA
:100100002297FE010E948D05C23CD107C9F70E94CB
:1001100072010C9491050C9400001CBC6F72606518
:100120006CBD8DB58EB508956EBD0DB407FEFDCFC7
:100130008EB508956EBD442321F0842F90E00E9477
:10014000EB010DB407FEFDCF8EB508958DE061E0A3
:100150000E9433028BE061E00E9433028CE060E099
:100160000E9433028AE061E00E9433021CBC80E5F9
:100170008CBD8DB58EB5089584E191E00E94A600F6
:100180000895EF92FF920F931F9303EA11E0C801C5
:1001900060E071E00E94150484E1E82E81E0F82E11
:1001A000C70161E0409109010E949A008093150106
:1001B000C70161E00E9494008091090140911501FE
:1001C00050E0480F511D4093150150E060E070E091
:1001D000C8012AE030E00E94F304C80160E20E94F6
:1001E0000D04C80163E071E00E941504C70161E0DD
:1001F000409109010E949A0080931501C70161E0B6
:100200000E949400809109014091150150E0480F2F
:10021000511D4093150150E060E070E0C8012AE0F4
:1002200030E00E94F304C80160E20E940D04C8019E
:1002300066E071E00E941504C70161E04091090188
:100240000E949A0080931501C70161E00E9494000A
:10025000809109014091150150E0480F511D4093D4
:10026000150150E060E070E0C8012AE030E00E9433
:10027000F304C8010E941D046CE271E080E090E08C
:100280000E94C1011F910F91FF90EF9008950F936D
:100290001F93DF93CF930F92CDB7DEB783EA91E040
:1002A00040E05BE460E070E00E949002CE010196C5
:1002B0000E94A60004E111E0C80160E00E948D00E8
:1002C000C80161E0409109010E949A00C80161E003
:1002D000409109010E949A000F90CF91DF911F91E8
:1002E0000F9108950E94F9010E9447010E94C100E8
:1002F000FDCF1F920F920FB60F9211242F933F93B1
:100300008F939F93AF93BF9380911A0190911B019C
:10031000A0911C01B0911D0130911E010196A11DFB
:10032000B11D232F2D5F2D3720F02D570196A11DD4
:10033000B11D20931E0180931A0190931B01A0937D
:100340001C01B0931D018091160190911701A0919D
:100350001801B09119010196A11DB11D80931601DC
:1003600090931701A0931801B0931901BF91AF9119
:100370009F918F913F912F910F900FBE0F901F90E3
:100380001895EF92FF920F931F937B018C018FB70B
:10039000F89440911A0150911B0160911C017091D9
:1003A0001D018FBF2FB7F89480911A0190911B0106
:1003B000A0911C01B0911D012FBF841B950BA60BB2
:1003C000B70BE816F9060A071B0760F71F910F9194
:1003D000FF90EF900895019759F0FC01EE0FFF1F79
:1003E000EE0FFF1F32978FB7F8943197F1F78FBF59
:1003F0000895789484B5826084BD84B5816084BD9D
:1004000085B5826085BD85B5816085BDEEE6F0E08D
:10041000808181608083E1E8F0E080818260808378
:10042000808181608083E0E8F0E08081816080836A
:10043000E1EBF0E0808184608083E0EBF0E080819C
:1004400081608083EAE7F0E080818460808380813E
:1004500082608083808181608083808180688083E6
:100460001092C1000895282F30E0C90186569F4F91
:10047000FC0194912A573F4FF9018491882391F010
:10048000E82FF0E0EE0FFF1FE859FF4FA591B49160
:10049000662329F48C91909589238C9308958C91EF
:1004A000892B8C9308951F920F920FB60F921124EF
:1004B0002F933F934F935F936F937F938F939F936C
:1004C000AF93BF93EF93FF934091C600E0919F01DC
:1004D000F091A001CF01019660E870E00E9427052D
:1004E0009C018091A1019091A2012817390739F050
:1004F000E15EFE4F40833093A00120939F01FF9166
:10050000EF91BF91AF919F918F917F916F915F918B
:100510004F913F912F910F900FBE0F901F90189504
:100520005F926F927F928F929F92AF92BF92CF9283
:10053000DF92EF92FF920F931F93CF93DF93EC0123
:100540003A014B01413482E458078FE0680780E0AC
:1005500078070CF07FC060E874E88EE190E0A401B9
:1005600093010E945C052150304040405040CA0138
:10057000B90122E030E040E050E00E945C05590102
:100580006A01A6019501209530954095509594E01B
:10059000220F331F441F551F9A95D1F760E074E274
:1005A00084EF90E00E945C05CA01B9012FEF30E0B2
:1005B00040E050E00E940805A40193010E945C0500
:1005C000C90181509F4F181619061CF4522E5A94D7
:1005D00003C055245394521A60E079E08DE390E013
:1005E000A40193010E945C052150304040405040DE
:1005F000CA01B90122E030E040E050E00E945C0511
:10060000209530954095509583E0220F331F441F6D
:10061000551F8A95D1F760E074E284EF90E00E9464
:100620005C05CA01B9012FEF30E040E050E00E94C4
:100630000805A40193010E945C05C90181509F4FE8
:10064000181619061CF4822F815002C081E0821B0B
:10065000851500F5E885F98581E090E00A8802C0FB
:10066000880F991F0A94E2F7808360E079E08DE3B8
:1006700090E0A40193010E945C052150304040406D
:100680005040CA01B90122E030E040E050E00E9451
:100690005C0504C0E885F98510829501EC81FD8137
:1006A0003083EE81FF812083EA85FB85208141E054
:1006B00050E0CA010E8402C0880F991F0A94E2F725
:1006C000282B2083EA85FB852081CA010F8402C084
:1006D000880F991F0A94E2F7282B2083EA85FB856F
:1006E0008081088802C0440F551F0A94E2F7842BCA
:1006F0008083DF91CF911F910F91FF90EF90DF905A
:10070000CF90BF90AF909F908F907F906F905F90B1
:100710000895FC01A085B18521898C9190E0022E7D
:1007200002C0959587950A94E2F780FFF6CF04847E
:10073000F585E02D608308958EE091E09093A4010B
:100740008093A3018FE191E09093A6018093A5018E
:1007500085EC90E09093A8018093A70184EC90E051
:100760009093AA018093A90180EC90E09093AC0152
:100770008093AB0181EC90E09093AE018093AD014A
:1007800086EC90E09093B0018093AF0184E0809379
:10079000B10183E08093B20187E08093B30185E0EB
:1007A0008093B40181E08093B50108950F931F9366
:1007B000CF93DF938C01EB0109C02196D801ED9115
:1007C000FC910190F081E02DC801099568816623B4
:1007D000A1F7DF91CF911F910F910895EF92FF92B2
:1007E0000F931F93CF93DF938C017B01EA010CC021
:1007F000D7016D917D01D801ED91FC910190F081BF
:10080000E02DC80109952197209791F7DF91CF91AD
:100810001F910F91FF90EF900895DC01ED91FC91F5
:100820000190F081E02D09950895DC01ED91FC9196
:100830000280F381E02D099508950F931F938C0199
:10084000DC01ED91FC910190F081E02D6DE00995C6
:10085000D801ED91FC910190F081E02DC8016AE092
:1008600009951F910F9108952F923F924F925F9299
:100870006F927F928F929F92AF92BF92CF92DF92B0
:10088000EF92FF920F931F93DF93CF93CDB7DEB715
:10089000A0970FB6F894DEBF0FBECDBF1C016A0152
:1008A0007B01411551056105710549F4DC01ED91AC
:1008B000FC910190F081E02D60E3099554C08824FB
:1008C00099245401422E55246624772401E010E037
:1008D0000C0F1D1F080D191DC701B601A3019201C0
:1008E0000E943A05F80160830894811C911CA11CA8
:1008F000B11CC701B601A30192010E943A05C901CA
:10090000DA016C017D01C114D104E104F104F1F6B6
:1009100081E0E82EF12CEC0EFD1EE80CF91C3E01E6
:100920000894611C711CD501C4010197A109B1098A
:100930006C01C818D90814C0F601EE0DFF1D6081C6
:100940006A3010F4605D01C0695CD101ED91FC91E9
:100950000190F081E02DC10109950894E108F108AA
:100960006E147F0449F7A0960FB6F894DEBF0FBE51
:10097000CDBFCF91DF911F910F91FF90EF90DF904E
:10098000CF90BF90AF909F908F907F906F905F902F
:100990004F903F902F900895EF92FF920F931F93E7
:1009A000CF93DF93EC017A018B0177FF0FC0E881D1
:1009B000F9810190F081E02D6DE209951095009587
:1009C000F094E094E11CF11C011D111DCE01B80151
:1009D000A7012AE00E943404DF91CF911F910F916B
:1009E000FF90EF900895DC012115310541F4ED9160
:1009F000FC910190F081E02D642F099508952A3033
:100A0000310519F40E94CC0408950E94340408951D
:100A1000629FD001739FF001829FE00DF11D649FE2
:100A2000E00DF11D929FF00D839FF00D749FF00D6E
:100A3000659FF00D9927729FB00DE11DF91F639F0F
:100A4000B00DE11DF91FBD01CF011124089597FBE1
:100A5000092E07260AD077FD04D049D006D0002001
:100A60001AF4709561957F4F0895F6F790958195EA
:100A70009F4F0895A1E21A2EAA1BBB1BFD010DC0BA
:100A8000AA1FBB1FEE1FFF1FA217B307E407F5073E
:100A900020F0A21BB30BE40BF50B661F771F881F1A
:100AA000991F1A9469F760957095809590959B01B0
:100AB000AC01BD01CF01089597FB092E05260ED08C
:100AC00057FD04D0D7DF0AD0001C38F4509540956C
:100AD000309521953F4F4F4F5F4F0895F6F7909512
:100AE0008095709561957F4F8F4F9F4F0895AA1BFA
:100AF000BB1B51E107C0AA1FBB1FA617B70710F009
:100B0000A61BB70B881F991F5A95A9F7809590953A
:100B1000BC01CD010895EE0FFF1F0590F491E02D6B
:060B20000994F894FFCFD8
:100B2600583D00593D005A3D000A00000000890367
:040B3600D603EE03F1
:00000001FF
